:100000006728672867286728F400030E8301F50036
:100010000A08F6000408F3008A018B1821280B1D3A
:100020005D280B1137080F3C031C1928B70A101460
:100030005D28B701C81D5D286400481A5D2848176F
:100040005D28481186184815C81A5A28B301B2010C
:10005000B1010A3049183E286430C9183E280330DF
:10006000B100E83049193E282730B1001030C919D5
:100070003E280130B2008630B100A030B0004819EF
:100080004C28B009B109B209B309B00F4C28B10F1F
:100090004C28B20F4C28B30A3008EB07310803187C
:1000A000310FEA0732080318320FE9073308031843
:1000B000330FE707B701C814C8158B1076088A00FC
:1000C00073088400750E8300F40E740E0900831209
:1000D00003138501860107309F008316F8308500E1
:1000E000033086000730810000308C008312F4302A
:1000F0008B0004309000043092007E28D024013020
:100100003E26B900B91F051ED322BC30E424E124E9
:10011000D501CD30E4245508583C031D85285130C5
:10012000F0000630F2003C26B524F20B93280A308A
:10013000F200FA30E925F20B99286922DE24051530
:10014000C801A8254F25AF251A26F225B618B729CC
:10015000361ACE283619C521B619F42136180C22C4
:10016000B61AFF21C818A228481FBB283F304A18DA
:100170004630B2224813851DC0208519C720A52806
:10018000361B08003617C814CA1C0800F429361F8D
:1001900008003613C814CA1C0800F429C816013018
:1001A000D400D824DE245330E424E1246230D4186F
:1001B000713054198030D4198F30541AE830D41A61
:1001C0009E30E4241A26F225B618F628C81CE32827
:1001D000C8100310481DF128D40D0130541BD40061
:1001E000D528D40C20300318D400D528D41A2C2AB2
:1001F000541A7129D4195B2954195729D4182F2955
:10020000361B2A2939144816C812DE244D30F00056
:100210003E26E7003C26E9003C26EA003C26EB00AF
:10022000F5244F25DD25F225C8181029B618B72169
:10023000361E13296708DA00F1004D30F00022263F
:100240006908DB0020266A08DC0020266B08DD0038
:1002500020267822D8244812C812C815A22858305F
:10026000332158304F294816C812E701E901F00040
:100270003E26EA003C26EB000130C900DE24742350
:10028000F524822476248B249B245F25DD25F2250A
:10029000C8183F29B618B721361E47290800F000B4
:1002A0006A08F10022266B08202678222A295A3073
:1002B00033215A304F294816C816DE24B0304A1967
:1002C000B630E424C810C81C6B294A1969294A159C
:1002D0005D294A115D29F225361E63290422DE219B
:1002E0002A2939144816C816DE249022470893227A
:1002F0008030AA242B30C71F2D30B5247F30470211
:10030000E30003188529E309E30AE201E10164300F
:10031000E302031C8D29E10A8829E3070A30E3027E
:10032000031C9429E20A8F29E3076108303EB524B3
:100330006208303EB5246308303EB5243030B52421
:100340003030B524D830E4244F25F225361AB029B0
:10035000C81CA529C810481DC7034819C70A762913
:100360004708F1005C30F000222678222A29C814C0
:100370000310490D1F39C90002300319C9000130AB
:10038000491AC900481A08002A29003038180730CD
:10039000B8180E3038191530B8191C30381A2330F7
:1003A000B81A2A30381B3130B81B3830B22203104B
:1003B000380801300319B800031DB80D0030381893
:1003C0000730B8180E3038191530B8191C30381AE3
:1003D0002330B81A2A30381B3130B81B3830F000BF
:1003E000C622C814C81508004A1CF9294A1046300C
:1003F000FB294A143F30B222042278220800CA1C8A
:10040000032ACA10042ACA145130F0004A08F10025
:100410002226C814C8150800C814C815391C132A88
:10042000B901B914172AB91C1E2AB9013915583057
:10043000F0003E26C5003C26C6000800391D292ACA
:10044000B901B9155A30F0003E26C5003C26C60059
:100450000800B901391408004816DE24F22451308E
:10046000F0008030C40070083C26C3004A2A4819B6
:10047000C30A481DC3035C30430230300318C30075
:10048000303043025B30031CC30043085B3C203028
:10049000031D4308B5244408AA24C810F225C8182F
:1004A000372A361A632AB61C4E2A43085B3C203092
:1004B000031D4308F1002226440AC400AA2444086C
:1004C000853C0318332AD8246430E9254812C81221
:1004D00085284D30F0003E26DA003C26DB003C2625
:1004E000DC003C26DD0051303E26CA00CA1BCA0192
:1004F0003F304A184630C3223808813C031CB801FB
:10050000B91F842A0130B900C91F882A0230493036
:100510005830B9195A30F0003E26C5003C26C600B6
:100520005C303E26C700CF002030A4000130A5007B
:10053000A601F030AB008830AC005B30AD00240881
:10054000AB0725080318250FAC0726080318260F4C
:10055000AD07CF0B9F2A2B08D8002C08D7002D08F9
:10056000D6000800F0003808F100222639082026BD
:100570004908202667082026690820266A082026C0
:100580006B0820260800F0003E26B8003C26B90083
:100590003C26C9003C26E7003C26E9003C26EA0050
:1005A0003C26EB000800DE242D30E424B8010130A5
:1005B000B9000430C90024230301B222D101B80AD2
:1005C000242307305107D100B2220310B80D031CB9
:1005D000E02AB801242307305107D100B2220730A6
:1005E0005107D100B2220030F1004D30F000222638
:1005F0004D302026D1302026E03020260530F10075
:100600005830F0002226DC3020260230F1005A302B
:10061000F0002226EE3020267F30F1005C30F00022
:1006200022264C30F1005230F00022265530202690
:1006300035302026443020264A30202656302026C9
:10064000FA30E925DE240800E7011B30E9007730A5
:10065000EA004030EB00381C332B3530E9006730BE
:10066000EA00E030EB00B81C3B2B6A30E900CF30E9
:10067000EA00C030EB00381D432B9A30E9004430CB
:10068000EA003030EB00B81D4B2BD530E9009F302D
:10069000EA008030EB00381E552B0130E7001330A4
:1006A000E900B230EA002030EB00B81E5F2B0130C9
:1006B000E7004030E9006F30EA004030EB00381FBF
:1006C000692B0130E7007B30E900CA30EA00903046
:1006D000EB00B81F08000130E700BA30E9008130B4
:1006E000EA004030EB000800E71F7B2BE701E9013F
:1006F000EA01EB0108006A080F3C031808000F30FC
:10070000EA00A030EB000800A301A201B301270D0D
:10071000A20D2D08A2022E08031C2E0FA302030116
:10072000031C0130B302A70D0730B400270DA20D42
:10073000A30DB30D2D08271CA72BA2022E08031C06
:100740002E0FA3020301031C0130B302B02BA2073A
:100750002E0803182E0FA307030103180130B30757
:10076000A70DB40B962B260DA20DA30DB30D2D08CE
:10077000271CC42BA2022E08031C2E0FA302030168
:10078000031C0130B302CD2BA2072E0803182E0F35
:10079000A307030103180130B307A60D0730B40007
:1007A000260DA20DA30DB30D2D08261CE12BA202D0
:1007B0002E08031C2E0FA3020301031C0130B302F9
:1007C000EA2BA2072E0803182E0FA3070301031814
:1007D0000130B307A60DB40BD02B250DA20DA30D30
:1007E000B30D2D08261CFE2BA2022E08031C2E0F73
:1007F000A3020301031C0130B302072CA2072E0839
:1008000003182E0FA307030103180130B307A50D2A
:100810000730B400250DA20DA30DB30D2D08251C26
:100820001B2CA2022E08031C2E0FA3020301031C83
:100830000130B302242CA2072E0803182E0FA307A1
:10084000030103180130B307A50DB40B0A2C240DC6
:10085000A20DA30DB30D2D08251C382CA2022E08C5
:10086000031C2E0FA3020301031C0130B302412C11
:10087000A2072E0803182E0FA30703010318013047
:10088000B307A40D0730B400240DA20DA30DB30DC2
:100890002D08241C552CA2022E08031C2E0FA30287
:1008A0000301031C0130B3025E2CA2072E080318BB
:1008B0002E0FA307030103180130B307A40DB40BD7
:1008C000442C2418692C2D08A2072E0803182E0F7B
:1008D000A3070034EF09EE09ED09EC09EF0F08005A
:1008E000EE0F0800ED0F0800EC0A0800C209C1096C
:1008F000C009BF09C20F0800C10F0800C00F0800DF
:10090000BF0A08006B08C2006A08C1006908C0007D
:100910006708BF0008005D08EF005C08EE005B0898
:10092000ED005A08EC0008004608EF004508EE000C
:10093000ED01EC0108006F08C2076E0803186E0F86
:10094000C1076D0803186D0FC0076C0803186C0F02
:10095000BF070800BD00C1243D0EC1243D08033C73
:100960000530031CB92CE9250800BD00CC243D0E40
:10097000CC242030BD006400BD0BBB2C061103113C
:100980000800F03986008615000000000000000015
:100990000000000086110800F03986000615C32CFF
:1009A0000330DE000530E9252030AD24DE0BD22CEB
:1009B0002830AA240C30AA240630AA240130AA2404
:1009C0000800C030AA240800BB000730DE005E0823
:1009D0008A003B080027D507BB0AFF390319080026
:1009E000B524E72C0E30AA2408006B08A4006A087E
:1009F000A5006908A6006708A7000430AA248D3066
:100A0000AA2448100330F20042252E304818203026
:100A1000B5240330F20042252E3048182030B5248A
:100A20002B254818192DAE010A30AD008423303033
:100A30002207B5242B254818232DAE010A30AD001E
:100A4000842330302207B5240630AA248E30AA240D
:100A5000D830E42408002030481808002708031D77
:100A600008002608031D08002508031D08002408A7
:100A7000093C031C080020304818080030302407C7
:100A8000481408002B2548184B2DAE010A30AD0044
:100A9000842330302207B524F20B422D08008B133B
:100AA000822439185F2D8B244A196A249B24BF1B8A
:100AB00076249424B91C6A249B24BF1B7624E50168
:100AC000EF01EE01ED01EC012030BE002230CB0041
:100AD0005608CC005708CD005808CE0003104E1C15
:100AE000882D4208EF07031C7A2DEE0F7A2DED0FAB
:100AF0007A2DEC0A4108EE07031C812DED0F812DA4
:100B0000EC0A4008ED07031C862DEC0A3F08EC07B1
:100B1000EC0CED0CEE0CEF0CE50CCB0CCC0CCD0C76
:100B2000CE0CBE0B6E2D04303918361B0030EC0095
:100B30002830BE008B130511EC0CED0CEE0CEF0C05
:100B4000E50C031C0510031805140515BE0B9B2DA1
:100B5000051100008514000085108B1708008030F7
:100B6000AA24003038180530B8180A3038190F3068
:100B7000B8191430381A1930B81A1E30381B2330FF
:100B8000B81B2830E424F524E1244F30B91847304D
:100B900039194330B9194B30E424E030361FE430C2
:100BA000E4243E30E4247E30B52441304A184230FB
:100BB000B524DB30CA1CAA30E424F22449188C3056
:100BC000C9188B3049198930C9198830AA24C8102E
:100BD0000800BE00F830BD006400BD0BEC2DBE0B5C
:100BE000EA2D08004030B6050A30E925051A032E23
:100BF0000130B700640037080319022E051EFA2DD4
:100C0000B614032E3616851F3615051B122E01301D
:100C1000B700640037080319112E051F092EB615F9
:100C2000122EB616851E36146400851F142E851EDE
:100C3000142E08006400051E1A2E051F1A2E080027
:100C4000F100F00A0313831664009C18242E700828
:100C50009B0071089A001C158B138B1B2C2E553092
:100C60009D00AA309D009C148B171C110313831246
:100C70000A30E9258B170800F00A70086400031396
:0E0C800083169B001C141A080313831208002D
:100E000082073134363430346D3400343834303481
:100E10006D3420340034343430346D3420340034B4
:100E2000333430346D3420340034323430346D3463
:100E300020340034313437346D34203400343134CC
:100E400035346D3420340034313432346D34203450
:100E50000034313430346D3420340034443445347B
:100E60004634413455344C345434203456344134AF
:100E70004C34553445345334203420340034203439
:100E8000763466346F34003455345334423400348D
:100E90004C34533442340034433457342034003417
:100EA000473445344E340034533445345434553487
:100EB0005034203420342034203420342034203462
:100EC0002034203400343134293420344F34463433
:100ED0004634533445345434203449342E34463463
:100EE0002E3400343234293420344F3446344634DE
:100EF000533445345434203453345334423420343E
:100F000000343334293420344F3446344634533497
:100F1000453454342034433457342034203400349E
:100F200034342934203443344F344E345634453429
:100F30005234543449344F344E342034003436342F
:100F40002934203451345234413420342034203474
:100F500020342034203420342034203420342034F1
:100F600000344C344F342B344934463400344C3440
:100F70004F342D34493446340034563446344F34DB
:100F800020342D3420344434443453342034203439
:100F90002034763431342E34333400344C345534E8
:100FA000353444344A34563420342F342F342034EA
:100FB000003448347A3400342034533470346C3480
:100FC00000342034543478340034203452347834AB
:100FD0000034353429342034433441344C342E34F5
:100FE00020345834543441344C34203420340034C8
:02400E00543F1D
:00000001FF
